:020000040800F2
:1000000000000220C14C0008ED4B0008EF4B000837
:10001000F14B0008F34B0008F54B0008000000000E
:10002000000000000000000000000000F74B000886
:10003000F94B000800000000FB4B0008FD4B0008D6
:10004000114D0008114D0008114D0008114D000818
:10005000114D0008114D0008114D0008114D000808
:10006000114D0008114D0008114D0008114D0008F8
:10007000114D0008114D0008114D0008114D0008E8
:10008000114D0008114D0008114D0008054C0008E5
:10009000114D0008114D0008114D0008114D0008C8
:1000A000114D0008114D0008114D0008114D0008B8
:1000B000114D0008114D0008114D0008114D0008A8
:1000C000114D0008114D0008114D0008114D000898
:1000D000114D0008114D0008114D0008114D000888
:1000E000114D0008114D0008114D0008114D000878
:1000F000114D0008114D0008114D0008114D000868
:10010000114D0008114D0008114D0008114D000857
:10011000114D0008114D0008114D0008114D000847
:10012000114D0008114D0008114D0008114D000837
:10013000114D00080000000000000000114D0008F3
:10014000114D0008114D0008114D0008114D000817
:10015000114D0008114D0008114D0008114D000807
:10016000114D0008114D0008114D0008114D0008F7
:10017000114D0008114D0008114D0008000000004D
:10018000114D0008114D0008114D0008114D0008D7
:10019000114D0008114D0008114D0008114D0008C7
:1001A000114D0008114D0008114D0008114D0008B7
:1001B000114D0008114D0008114D0008114D0008A7
:1001C000114D0008114D0008000000000000000063
:1001D0000000000000000000114D000800000000B9
:1001E000000000000000000000000000000000000F
:1001F0000000000000000000114D0008114D000833
:10020000114D0008114D000800000000114D0008BC
:10021000114D0008114D0008114D0008114D000846
:10022000114D0008114D0008114D0008000000009C
:10023000114D0008114D000800000000114D00088C
:10024000114D0008114D0008114D0008114D000816
:10025000114D0008114D0008114D0008114D000806
:10026000114D0008114D0008114D0008114D0008F6
:10027000114D0008114D0008114D0008000000004C
:10028000114D0008114D000800000000114D00083C
:1002900000000000114D0008114D00080000000092
:0C02A00000000000114D0008114D000886
:1002AC0010B5054C237833B9044B13B10448AFF3A4
:1002BC0000800123237010BD1000002000000000FE
:1002CC00884D000808B5034B1BB103490348AFF335
:1002DC00008008BD0000000014000020884D0008BC
:1002EC002DE9F0438BB005AD0024059406940794DA
:1002FC0008940994414BD3F8402142F08002C3F892
:10030C004021D3F8402102F080020192019AD3F8E7
:10031C00402142F00402C3F84021D3F8402102F0FE
:10032C0004020292029AD3F8402142F00102C3F86F
:10033C004021D3F8402102F001020392039AD3F832
:10034C00402142F00202C3F84021D3F8403103F0BF
:10035C0002030493049BDFF8AC802246F421404650
:10036C0001F066FCDFF8A090224648F204014846F2
:10037C0001F05EFC224E22464FF40941304601F05A
:10038C0057FCF423059301270697079408942946F4
:10039C00404601F03DFB40F2CB6305930694079475
:1003AC002946304601F034FB42F2C34305930694D0
:1003BC0007942946484601F02BFB48F204030593A9
:1003CC000697079408942946484601F021FB4FF400
:1003DC0000730593069407942946404601F018FBD8
:1003EC004FF4094305930697079408942946304621
:1003FC0001F00EFB0BB0BDE8F08300BF00440258C7
:10040C0000000258000802580004025872B6FEE7B9
:10041C0008B51648164B036000238360C360037451
:10042C004374837402224261012282611F21C161E3
:10043C000821016242628262C2620263436320212C
:10044C008163C36310220264042242648364C26425
:10045C00036542658365C36501664366826600F089
:10046C00EBFF00B908BDFFF7D1FF00BF88010020EA
:10047C0000A0004000B58DB00023079308930993AA
:10048C000A930B93039304930593069300930193A0
:10049C0002932348234A026043F67F6242608360E2
:1004AC004FF6FF72C26003614361836104F088F907
:1004BC0000282BD10423079350230893002309937E
:1004CC000A930B9307A9164804F010FB00BB0022FB
:1004DC000392012304930592069203A9104804F099
:1004EC00E9F9B8B9022303930493042203A90C4835
:1004FC0004F0E0F980B900230093029369460848A0
:10050C0004F01EFB50B90DB05DF804FBFFF77EFF45
:10051C00FFF77CFFFFF77AFFFFF778FFFFF776FF17
:10052C002C0000200040014008B51348134B036019
:10053C004FF480034360002383600322C260036195
:10054C0043614FF000528261C36103624362836274
:10055C00C3624FF0804242638363C36303644364AA
:10056C008364C36403654365836503F05FFF00B96F
:10057C0008BDFFF74BFF00BF000100200030014019
:10058C0008B51248124B03604FF4800343600023FC
:10059C0083600322C260036143618361C3610362B0
:1005AC0043628362C3624FF0804242638363C363DE
:1005BC00036443648364C36403654365836503F028
:1005CC0035FF00B908BDFFF721FF00BF7800002000
:1005DC000038004000B58BB00023079308930993B3
:1005EC0000930193029303930493059306931D4880
:1005FC001D4A026043608360C3600422026103757C
:10060C00437501228261037743628362C362036391
:10061C00436380F8383000F029FCE0B900230793DD
:10062C0007A9104800F01EFDB8B9104B0093062323
:10063C0001930023029340F2FF720392042204926E
:10064C0005938DF819306946064800F07BF930B9EE
:10065C000BB05DF804FBFFF7D9FEFFF7D7FEFFF7F1
:10066C00D5FE00BF8C020020002002400004002AAE
:10067C0000B589B00023019302930393049305936F
:10068C00069307931848194A026043608360C3605D
:10069C000422026103754375012282610377436270
:1006AC008362C3620363436380F8383000F0DEFB7F
:1006BC00A8B90F4B019306230293002303930D4A11
:1006CC0004920422059206938DF81D300DEB020165
:1006DC00054800F037F920B909B05DF804FBFFF7C5
:1006EC0095FEFFF793FE00BF280200200021024078
:1006FC000004002A0000FF4700B59DB04C220021E9
:10070C0009A804F000FB2022002101A804F0FBFA48
:10071C00234B4FF0FF32C3F8B020022001F05EFCF7
:10072C00002300931F4B9A6922F440429A619B6903
:10073C0003F440430093009B1A4B9B6913F4005F36
:10074C00FAD0012209924FF480330A9302231293B8
:10075C0013931492082215921693179318930C2343
:10076C00199300231A931B9309A801F061FC90B90B
:10077C003F230193032302930023039304930593D4
:10078C00069307930893022101A802F07DF820B983
:10079C001DB05DF804FBFFF739FEFFF737FE00BF15
:1007AC00004402580048025830B5B1B0C0252A4662
:1007BC000021684604F0A7FA4FF408220023CDE983
:1007CC00002301230293082303930323049305932B
:1007DC000223069307954FF000531E93684602F0D0
:1007EC00D9FA08B931B030BDFFF710FE08B500F0EA
:1007FC003BF8FFF781FFFFF7D7FFFFF771FDFFF71E
:10080C0007FEFFF737FEFFF78FFEFFF7B9FEFFF786
:10081C00E1FEFFF72DFFFEE7104B1B780BB9012013
:10082C00704710B504464FF47A70B0FBF3F30C4AE2
:10083C001068B0FBF3F000F001FD68B90F2C01D982
:10084C0001200AE0002221464FF0FF3000F0E2FCCC
:10085C00044B1C60002000E0012010BD00000020B3
:10086C000C0000200400002010B5032000F0C0FC98
:10087C0001F00EFF0F498B69C3F303230E4AD35CBF
:10088C0003F01F03D8408B6903F00F03D35C03F014
:10089C001F0320FA03F3094A1360094B18600F2059
:1008AC00FFF7BAFF10B10124204610BD044601F039
:1008BC00C5F9F9E700440258EC4D00080800002087
:1008CC000C000020034B1B78034A11680B44136087
:1008DC00704700BF00000020F0020020014B186898
:1008EC00704700BFF002002010B430300B0A9B00A0
:1008FC0003F00C03C45801F01F014FF01F0C0CFA4D
:10090C0001FC24EA0C0CC2F384628A404CEA020219
:10091C00C2505DF8044B704710B414304B0E9B0062
:10092C0003F00403C458C1F304514FF0070C0CFA44
:10093C0001FC24EA0C0C8A404CEA0202C2505DF81D
:10094C00044B7047F0B583B00023019390F85030FE
:10095C00012B00F0FA8104460D46012380F850303B
:10096C000268936813F0040F09D0436D43F0200321
:10097C0043650120002384F8503003B0F0BD0B68B0
:10098C00002B0ADBC3F31301002939D1C3F38463B1
:10099C0001219940D3690B43D3612A6869682068A7
:1009AC00FFF7A2FF2068866816F0040600D0012627
:1009BC00836813F0080F00D176B321688B6813F0AD
:1009CC00010F40F0BE812B68E868D1F8C020C3F35A
:1009DC00130622EA060200F01806A148F040034074
:1009EC00C3F313031343C1F8C030EA689D4B9A421A
:1009FC0000F08F802B68002BC0F236810020B9E705
:100A0C0093FAA3F333B1B3FA83F303F01F03012179
:100A1C009940BFE72023F8E7AA682968FFF77CFF15
:100A2C002368DA6812F0100F31D16A69D968C1F302
:100A3C00820149008A402F69042F36D02868603320
:100A4C0053F8271001F0004100F0F84002430A432C
:100A5C0043F82720236828696A7E012A1FD0324672
:100A6C00603353F8201021F000410A4343F8202052
:100A7C00206829692B7E012B14D0026922F4F042E4
:100A8C0001F01F0306FA03F31343036195E76A6948
:100A9C00D968890801F0040149008A40CBE74FF07E
:100AAC000042DDE74FF40066E7E71A6E02F0F84209
:100ABC002968B2EB816F1DD02268536E03F0F843A6
:100ACC002968B3EB816F1AD02268936E03F0F84358
:100ADC002968B3EB816F17D02268D36E03F0F8430B
:100AEC002968B3EB816F7FF468AFD36E23F00043BA
:100AFC00D36662E71A6E22F000421A66DCE7536E88
:100B0C0023F000435366DFE7936E23F000439366B4
:100B1C00E2E720682B68C3F3130626BB9A0E01325A
:100B2C0002F01F02092A8CBF00220122002A51D098
:100B3C0046BB990E0131890601F0F84176BB9F0E38
:100B4C00013707F01F070122BA401143A6BB9B0EC9
:100B5C00013303F01F0303EB43031B051943AA687E
:100B6C00FFF7DAFE46E793FAA3F24AB1B2FA82F241
:100B7C00013202F01F02092A8CBF00220122D5E7A4
:100B8C002022F5E793FAA3F131B1B1FA81F10131E9
:100B9C00890601F0F841D1E72021F8E793FAA3F296
:100BAC0042B1B2FA82F2013202F01F02012707FAB7
:100BBC0002F2CAE72022F6E793FAA3F343B1B3FAA1
:100BCC0083F3013303F01F0303EB43031B05C5E75A
:100BDC002023F6E7CEB9990E0131890601F0F841D0
:100BEC00FEB99F0E013707F01F070122BA401143CF
:100BFC002EBB9B0E013303F01F0303EB43031E3B81
:100C0C001B0543F000731943A9E793FAA3F131B123
:100C1C00B1FA81F10131890601F0F841E0E72021B8
:100C2C00F8E793FAA3F242B1B2FA82F2013202F07F
:100C3C001F02012707FA02F2D9E72022F6E793FAFE
:100C4C00A3F35BB1B3FA83F3013303F01F0303EB9C
:100C5C0043031E3B1B0543F00073D4E72023F3E74B
:100C6C00FFFF0F000000FF47394A916801F0E07563
:100C7C00A2F54072926812F0010200D001223548B0
:100C8C00806810F0010F56D1002A54D1324A934299
:100C9C0007D0324A934228D0314A934238D00020B0
:100CAC0068E611F4000FF4D122682A4B9A4201D065
:100CBC0000205FE645F4000325498A6822F0E072C3
:100CCC0013438B60274B1B689B09274AA2FB03230A
:100CDC009B0901335B00019302E0019B013B0193F3
:100CEC00019B002BF9D1002044E611F0807FD3D179
:100CFC002268184B9A4201D000203BE645F08073E5
:100D0C0013498A6822F0E07213438B60002031E6AD
:100D1C0011F4800F17D122680E4B9A4201D000209B
:100D2C0028E645F480030A498A6822F0E0721343EE
:100D3C008B6000201EE6636D43F020036365012089
:100D4C0018E6002016E6002014E6022015E600BF87
:100D5C000023024000210240000084CB0040C0BAB6
:100D6C000000B8CF0C000020632D3E0510B50446E2
:100D7C003A4B9B6813F4403F19D001F0CFFE6368E7
:100D8C00B3F5003F05D0B3F5403F0ED0B3F5803F2F
:100D9C0002D11B0CB0FBF3F0314B984241D82268C6
:100DAC00936823F44073936010BD8008F4E74FF40C
:100DBC000020002103F02AF86368B3F5101F2CD033
:100DCC0021D8B3F5E01F26D004D9B3F5001FE3D129
:100DDC004009E1E7B3F5801F10D009D8B3F5002F17
:100DEC000CD0B3F5402F09D0B3F5802F06D0D3E744
:100DFC00B3F5A01F02D0B3F5C01FCDD19B0C5B0087
:100E0C00B0FBF3F0C8E7B3F5201F08D0B3F5301FE3
:100E1C00C2D1000AC0E70009BEE78009BCE7C009DF
:100E2C00BAE7104B984207D82268936823F44073B2
:100E3C0043F480739360B7E70B4B984207D8226852
:100E4C00936823F4407343F400739360ACE7226817
:100E5C00936843F440739360A6E700BF00230240FD
:100E6C0021BCBE0041787D0181F0FA0230B583B01F
:100E7C0000230193002800F0DF800446436DEBB1A2
:100E8C0023689A6812F0005F03D099686B4A0A4095
:100E9C009A6023689A6812F0805F1CD19968684A3E
:100EAC000A4042F080529A60664B1B689B09664A66
:100EBC00A2FB03239B090133019309E000F0D0FE50
:100ECC000023A36584F85030DAE7019B013B0193C2
:100EDC00019B002BF9D12268936813F0805F40F0DE
:100EEC008180636D43F010036365A36D43F00103D0
:100EFC00A3650125936813F0040300D00123616DF1
:100F0C0011F0100F40F09080002B40F08D80636D3D
:100F1C0023F4817343F002036365936813F0010FAC
:100F2C0012D14A4B9B6813F0010300D00123484AAD
:100F3C00926812F0010F07D133B9636845498A688A
:100F4C0022F47C1213438B60627D236B43EA4233A1
:100F5C00A2681343227F43EA0243012A44D0626A07
:100F6C0022B102F47872A16A0A4313432168C8685B
:100F7C00394A02401A43CA602268936813F004038A
:100F8C0000D00123916811F0080F1CD1DBB9217D31
:100F9C00E36A43EA8131D068304B03400B43D360A2
:100FAC0094F83830012B24D02268136923F0010304
:100FBC0013612268136923F07043616B0B43136157
:100FCC002046FFF7D3FEE368012B24D02268136B75
:100FDC0023F00F031363636D23F0030343F001034A
:100FEC00636526E0002585E7226A013A43EA42431D
:100FFC00B5E7206802691A4B1340E26B511E226C54
:10100C0042EA0142616C0A43A16C0A43134343F068
:10101C0001030361CDE721680B6B23F00F03A26979
:10102C00013A13430B63D6E7636D43F0100363651A
:10103C000125284603B030BD0125FAE7C0FFFF5F4C
:10104C00C0FFFF6F0C000020632D3E050020024006
:10105C00002102400023024003C0F0FFFCBFFFFF51
:10106C001EF800FC90F85020012A78D010B49BB0E8
:10107C000346012280F85020002216921792006835
:10108C00384A904231D000220192019A002A30D085
:10109C00926812F0040200D00122806810F0040F54
:1010AC0049D1002A47D10A6862B32F48826822F4DA
:1010BC0040424C68224382602A4A926812F0010234
:1010CC0000D001222948806810F0010F3FD1002A7E
:1010DC003FD1254CA068A2F572620240086889686D
:1010EC0001430A43A26000202AE002F580720192BB
:1010FC00CBE75A6D42F020025A65002283F850204B
:10110C00012020E018498A6822F440428A60154A7E
:10111C00926812F0010200D001221449896811F082
:10112C00010F18D1CAB910498868A2F57262024041
:10113C008A60002004E05A6D42F020025A650120BA
:10114C00002283F850201BB05DF8044B7047002040
:10115C00F6E70020F4E70020F2E70020F0E7022099
:10116C00704700BF002002400023024000210240D3
:10117C00002807DB00F01F02400901239340024ABC
:10118C0042F82030704700BF00E100E0002804DB8B
:10119C000901C9B2044B1954704700F00F00090142
:1011AC00C9B2024B1954704700E400E014ED00E0A2
:1011BC0000B500F00700C0F1070CBCF1040F28BF0C
:1011CC004FF0040C031D062B0FD9C31E4FF0FF3E2E
:1011DC000EFA0CF021EA000199400EFA03FE22EA05
:1011EC000E0241EA02005DF804FB0023EEE700006A
:1011FC000649CB6823F4E0631B041B0C000200F4CB
:10120C00E0600343024A1A43CA60704700ED00E0F5
:10121C000000FA0510B50446054BD868C0F302204F
:10122C00FFF7C6FF01462046FFF7B0FF10BD00BF19
:10123C0000ED00E008B5FFF79BFF08BD0138B0F1E9
:10124C00807F0BD24FF0E0235861054AF02182F8E1
:10125C0023100020986107221A6170470120704703
:10126C0000ED00E030B4416B0468D4F884306F4A70
:10127C00134043EA8103C4F884300468D4F8843002
:10128C0023F47F03856B43EA0543C4F88430836BF6
:10129C000B440468D4F88810114041EA8301C4F867
:1012AC0088100468D4F8881021F4FE01C56B41EA5B
:1012BC000541C4F88810C16B03EB41030468D4F8F2
:1012CC00A010114041EA8301C4F8A0100468D4F8BE
:1012DC00A01021F4FE01056C41EA0541C4F8A010F0
:1012EC00016C446C04FB01330468D4F8B010114059
:1012FC0041EA8301C4F8B0100468D4F8B01021F4AA
:10130C00FE01856C41EA0541C4F8B010816CC46CD7
:10131C0004FB01330468D4F8AC10114041EA83019A
:10132C00C4F8AC10016D446D04FB01330468D4F8AF
:10133C00F010114041EA8301C4F8F0100468D4F8AD
:10134C00F01021F47C11856D41EA0541C4F8F010D0
:10135C00816D03EB41030468D4F8C0100A4042EAE3
:10136C008303C4F8C0300268D2F8C03023F47C1375
:10137C00C16D43EA0143C2F8C0300268D2F8C030F4
:10138C0023F07C53016E43EA0163C2F8C030436B17
:10139C00274A1A449200C266836B02EB83030367ED
:1013AC00C16B03EBC1034367016C446C04FB01F19B
:1013BC0003EB81038367816CC46C04FB01F103EBC9
:1013CC008103C367016D446D04FB01F103EB8103E1
:1013DC00C0F88030816D03EBC103C0F88430816E9E
:1013EC00C46D01FB04FC03EB8C03C0F88830046E65
:1013FC0004FB01F103EB8103C0F890300D498B42E3
:10140C000DD9D0F89C3043F02003C0F89C30032356
:10141C0080F89830012007E0002342F8043BD0F814
:10142C0090309342F8D8002030BC70470300FFFF87
:10143C00002B0010FCD3004030B595B004464C2274
:10144C00A04901A803F08CFC002C00F03881236823
:10145C009D4A934220D094F898300BB3226893693C
:10146C0023F010039361FFF739FA054623689A6954
:10147C0012F0080F1AD0FFF731FA431B0A2BF5D9DB
:10148C00D4F89C3043F00103C4F89C30032384F857
:10149C009830012015B030BD03F580736360DAE736
:1014AC0084F89930204600F04BFCD7E79A6942F05B
:1014BC0001029A61FFF712FA054623689A6912F045
:1014CC00010F0FD1FFF70AFA401B0A28F5D9D4F8FF
:1014DC009C3043F00103C4F89C30032384F898300B
:1014EC000120D7E79A6942F002029A61237C012B12
:1014FC0040D02268936943F040039361637C012BD5
:10150C003ED02268936923F480439361A37C012B22
:10151C003CD02268936943F48053936122689369A9
:10152C0023F44073A1680B4393612268936923F001
:10153C00A40393612268136923F010031361E36819
:10154C00012B29D0002B2CD0022B00F09B80226881
:10155C00936943F0800393612268136943F010038D
:10156C001361E368032B1CD12268936943F02003B9
:10157C00936116E02268936923F040039361BDE701
:10158C002268936943F480439361BFE722689369AF
:10159C0023F480539361C1E72268936943F00403F9
:1015AC009361A3695A1EE369013B1B0243EA426340
:1015BC00226A013A13436269013A216843EA024301
:1015CC00CB61A368B3F5407F62D0236E33B1226840
:1015DC00D2F8C030616E0B43C2F8C030E36D226E9E
:1015EC00D3420DD02168D1F8C83023F00703A26E86
:1015FC0014A800EB820252F84C2C1343C1F8C830EB
:10160C00236C6BB12168D1F8BC3023F00703626CFA
:10161C0014A800EB820252F84C2C1343C1F8BC30D6
:10162C00A36C73B12168D1F8BC3023F07003E26C69
:10163C0014A800EB820252F84C2C43EA0213C1F8B6
:10164C00BC30236D73B12168D1F8BC3023F4E06356
:10165C00626D14A800EB820252F84C2C43EA022370
:10166C00C1F8BC302268184B9A4222D00023C4F82F
:10167C009430C4F89C30012384F898302046FFF74E
:10168C00F1FD07E72268936943F02003936188E733
:10169C00A36A013BE26A013A43EA0223226B013A54
:1016AC0043EA0213626A013A216843EA0243CB60BF
:1016BC008BE76268936823F003039360D6E70120FD
:1016CC00E8E600BFA04D000800A00040704770473E
:1016DC007047704770477047704770477047704746
:1016EC0070477047704770477047704770470000ED
:1016FC002DE9F04F83B00446904B1A695B69134097
:10170C0001939B07009303681A6D02F4704A5A6D9B
:10171C000AEA020A1A6D02F00F095A6D09EA020967
:10172C001A6D02F0F0085A6D08EA02081E6D06F0F8
:10173C0071565A6D16401F6D07F060775A6D174041
:10174C005D6DD3F850B015F4807F02D01BF4807F10
:10175C0064D115F4806F02D01BF4806F67D1009BAD
:10176C00002B74D1BAF1000F7ED1B9F1000F40F00B
:10177C008780B8F1000F40F08F8015F4006F03D014
:10178C001BF4006F40F0948015F4007F03D01BF421
:10179C00007F40F0988015F4002F03D01BF4002F2D
:1017AC0040F0A18015F4803F03D01BF4803F40F043
:1017BC00A58015F4802F03D01BF4802F40F0A98056
:1017CC0015F4003F0FD01BF4003F0CD023684FF4EE
:1017DC0000321A65594B00221A61D4F89C3043F040
:1017EC008003C4F89C30002F40F09E804EB12368DB
:1017FC001E65B20F514B1A61D4F89C303343C4F8B8
:10180C009C3022684E4B9A4200F09C80D4F89C305D
:10181C00002B40F0F98003B0BDE8F08F4FF48072DC
:10182C001A65464B00221A61FFF75AFF91E72368AD
:10183C00D3F8DC10D3F8E4204FF4806018653F4BEC
:10184C000020186111402046FFF746FF87E7236808
:10185C0000221A65019B03F00303384A13610099B7
:10186C002046FFF733FF7DE72368C3F850A04FEA0B
:10187C009A72324B1A6151462046FFF728FF74E7E3
:10188C002368C3F850904FEA99722C4B1A61494661
:10189C002046FFF71DFF6CE72368C3F850804FEA22
:1018AC009872264B1A6141462046FFF712FF64E7F7
:1018BC0023684FF400621A65204B00221A612046FF
:1018CC00FFF708FF60E72368D3F8D810D3F8E020BF
:1018DC004FF400701865194B002018611140204618
:1018EC00FFF7F9FE57E723684FF400221A65134BF4
:1018FC0000221A612046FFF7F0FE53E723684FF4ED
:10190C0080321A650D4B00221A612046FFF7E6FE65
:10191C004FE723684FF480221A65084B00221A61A6
:10192C002046FFF7DCFE4BE723681F65BA0F034B1D
:10193C001A6139462046FFF7D5FE57E700A800404C
:10194C0000A0004063689A6812F0030F3FF45EAF8A
:10195C00196A01F00F015A6A186A00F03008586AC7
:10196C0008EA00081F6A07F4C077586A07401E6A25
:10197C0006F4FC46586A06401D6A05F4F025586AC0
:10198C000540D3F82490D3F820A011401CD1B8F115
:10199C00000F1ED119F0400F02D01AF0400F20D1C9
:1019AC005FBB36B163681E62D4F89C303343C4F815
:1019BC009C30002D3FF42AAF63681D62D4F89C3034
:1019CC002B43C4F89C3021E719622046FFF78BFEAD
:1019DC00DDE76368C3F8208041462046FFF784FEAC
:1019EC00D8E76368D96BDA6B4020186202F03F02CB
:1019FC00090C2046FFF779FED2E763681F6239466F
:101A0C002046FFF773FECCE72046FFF76AFE02E79D
:101A1C00F0B583B000236BE085685E000324B4400E
:101A2C0025EA0405CC68B4402C438460456825EA5B
:101A3C000C054C68C4F300149C402C43446069E0D2
:101A4C00DD08083550F8254003F0070C4FEA8C0CE4
:101A5C004FF00F0E0EFA0CFE24EA0E0E0C6904FA6F
:101A6C000CF444EA0E0440F825406BE0092400E035
:101A7C00002404FA0EF42C430CF1020C694D45F8C9
:101A8C002C404FF0B0442568D44325EA02064F6839
:101A9C0017F4801F01D042EA05064FF0B0452E60C6
:101AAC006D6804EA05064F6817F4001F01D042EA7E
:101ABC0005064FF0B0456E60D5F8845004EA050673
:101ACC004F6817F4003F01D042EA05064FF0B045CD
:101ADC00C5F88460D5F880502C404E6816F4803FD1
:101AEC0001D042EA05044FF0B042C2F88040013305
:101AFC000A6832FA03F400F092804FF0010C0CFAF1
:101B0C0003FC1CEA0202F2D04C6804F00304013C12
:101B1C00012C81D94C6804F00304032C0CD0C4684C
:101B2C005D004FF0030C0CFA05FC24EA0C0C8C68DD
:101B3C00AC4044EA0C04C4604C6804F00304022C6E
:101B4C003FF47EAF04684FEA430E4FF0030C0CFADF
:101B5C000EFC24EA0C0C4C6804F0030404FA0EF49A
:101B6C0044EA0C0404604C6814F4403FBFD02E4C83
:101B7C00D4F8545145F00205C4F85451D4F85441EA
:101B8C0004F002040194019C4FEA930C0CF1020541
:101B9C00244C54F8255003F0030E4FEA8E0E0F24FC
:101BAC0004FA0EF425EA0405204CA0423FF460AF81
:101BBC0004F58064A04222D004F58064A04220D0B9
:101BCC0004F58064A0421ED004F58064A0421CD0B1
:101BDC0004F58064A0421AD004F58064A04218D0A9
:101BEC0004F58064A04216D004F58064A04214D0A1
:101BFC0004F58064A0423FF439AF0A2439E701248C
:101C0C0037E7022435E7032433E7042431E70524BE
:101C1C002FE706242DE707242BE7082429E703B038
:101C2C00F0BD00BF000400580044025800000258E8
:101C3C000AB18161704709048161704782B0074B1A
:101C4C00D3F8542142F00202C3F85421D3F8543192
:101C5C0003F002030193019B02B070470044025849
:101C6C0000B58BB000230593069307930893099353
:101C7C0003682E4A934205D02D4A93422CD00BB0C8
:101C8C005DF804FB2B4A136801331360012B15D04C
:101C9C00294BD3F8402142F00402C3F84021D3F879
:101CAC00403103F004030293029B012305930323A9
:101CBC00069305A92148FFF7ABFEE0E71E4BD3F8CE
:101CCC00382142F02002C3F83821D3F8383103F020
:101CDC0020030193019BDBE7164A13680133136061
:101CEC00012B14D0144BD3F8402142F00402C3F85A
:101CFC004021D3F8403103F004030493049B0323E5
:101D0C000593069305A90D48FFF782FEB7E70A4B2A
:101D1C00D3F8382142F02002C3F83821D3F83831F7
:101D2C0003F020030393039BDCE700BF0020024079
:101D3C0000210240F402002000440258000802581E
:101D4C0000B589B00023039304930593069307937E
:101D5C000268194B9A4202D009B05DF804FB174B8C
:101D6C00D3F84C2142F48072C3F84C21D3F84C21A7
:101D7C0002F480720192019AD3F8402142F00202DF
:101D8C00C3F84021D3F8403103F002030293029BC5
:101D9C004FF440730393022304930923079303A97D
:101DAC000748FFF735FE002211461320FFF732FAE1
:101DBC001320FFF73FFACFE700A000400044025881
:101DCC00000402582DE9F041BEB0044600213991BF
:101DDC003A913B913C913D91C02208A802F093FFAF
:101DEC0023685C4A934205D05B4A93424FD03EB085
:101DFC00BDE8F0814FF480520023CDE9082308A8F8
:101E0C0000F0C8FF00283FD1544BD3F8502142F4C6
:101E1C008052C3F85021D3F8502102F48052019221
:101E2C00019AD3F8402142F00102C3F84021D3F8C3
:101E3C00402102F001020292029AD3F8402142F0B2
:101E4C000202C3F84021D3F8403103F0020303939C
:101E5C00039B4FF03008CDF8E48002273A9700241A
:101E6C003B943C9405263D9639AD29463C48FFF7FA
:101E7C00CFFDCDF8E4803A973B943C943D962946AF
:101E8C003848FFF7C5FDB2E7FEF7C0FABCE74FF4E0
:101E9C0080520023CDE9082308A800F07BFF00281E
:101EAC0055D12E4BD3F8482142F48042C3F8482137
:101EBC00D3F8482102F480420492049AD3F84021CA
:101ECC0042F00402C3F84021D3F8402102F004028E
:101EDC000592059AD3F8402142F00202C3F8402142
:101EEC00D3F8402102F002020692069AD3F8402160
:101EFC0042F00102C3F84021D3F8403103F0010352
:101F0C000793079B0823399302273A9700243B94A5
:101F1C003C9405263D9639AD29461348FFF778FDCC
:101F2C004FF4A04339933A973B943C943D96294601
:101F3C000C48FFF76DFD4FF4805339933A973B945F
:101F4C003C943D9629460648FFF762FD4FE7FEF7A5
:101F5C005DFAA6E70030014000380040004402580A
:101F6C0000000258000402580008025800B589B05D
:101F7C000023039304930593069307930268144B71
:101F8C009A4202D009B05DF804FB124BD3F85021F1
:101F9C0042F48032C3F85021D3F8502102F480323D
:101FAC000192019AD3F8402142F00102C3F840217A
:101FBC00D3F8403103F001030293029B04230393F3
:101FCC0002220492079303A90348FFF721FDD9E7E6
:101FDC00004001400044025800000258134BDB68DB
:101FEC0013F0040F07D1114BDB6803F00703834296
:101FFC001AD00120704710B50C4AD36823F00703A0
:10200C000343D360FEF76AFC0446084B5B6813F489
:10201C00005F07D1FEF762FC001BB0F57A7FF4D9A4
:10202C00012000E0002010BD00207047004802583D
:10203C00002800F0118338B50446036813F0010F33
:10204C0029D0A14A136903F03803926A102B19D0D6
:10205C00182B13D06368B3F5803F43D0002B58D1B5
:10206C00994B1A6822F480321A601A6822F4801292
:10207C001A601A6822F480221A6038E002F0030217
:10208C00022AE7D1904B1B6813F4003F03D063681E
:10209C00002B00F0E382236813F0020F00F0A28003
:1020AC00894A1369926A13F0380374D0182B6FD0D5
:1020BC00E368002B00F0C38083490A6822F0190200
:1020CC0013430B60FEF70AFC05467F4B1B6813F0AD
:1020DC00040F40F0AB80FEF701FC401B0228F4D942
:1020EC000320C2E2784A136843F4803313606368B8
:1020FC00002B3ED0FEF7F2FB0546734B1B6813F426
:10210C00003FC8D1FEF7EAFB401B6428F5D9032039
:10211C00ABE2B3F5A02F10D0B3F5A81F1BD06A4BC0
:10212C001A6822F480321A601A6822F480221A602B
:10213C001A6822F480121A60D9E7634B1A6842F4C9
:10214C0080221A601A6822F480121A601A6842F40B
:10215C0080321A60CBE75C4B1A6842F480221A601A
:10216C001A6842F480121A601A6842F480321A60BB
:10217C00BDE7FEF7B3FB0546534B1B6813F4003F5A
:10218C0089D0FEF7ABFB401B6428F5D903206CE229
:10219C0012F0030F8CD14C4B1B6813F0040F03D0BF
:1021AC00E368002B00F05C82474A136823F01903A4
:1021BC00E1680B431360FEF791FB0546424B1B682D
:1021CC0013F0040F06D1FEF789FB401B0228F5D94A
:1021DC0003204AE23C4A536823F0FE43216943EA58
:1021EC0001635360236813F0100F51D0364A136902
:1021FC0003F03803926A082B39D0182B33D0E369DB
:10220C00002B6CD0304A136843F080031360FEF748
:10221C0065FB05462C4B1B6813F4807F56D1FEF7EB
:10222C005DFB401B0228F5D903201EE2264A5368A9
:10223C0023F0FE43216943EA01635360D2E7224A4B
:10224C00136823F001031360FEF748FB05461E4B91
:10225C001B6813F0040FC5D0FEF740FB401B02288F
:10226C00F5D9032001E202F00302012AC7D1164B73
:10227C001B6813F4807F03D0E369802B40F0F2815C
:10228C00114AD36823F07C53216A43EA0163D3607B
:10229C00236813F0080F4AD06369002B33D00A4A25
:1022AC00536F43F001035367FEF718FB0546064BCB
:1022BC005B6F13F0020F3AD1FEF710FB401B0228A4
:1022CC00F5D90320D1E100BF004402588C4AD368F1
:1022DC0023F07C53216A43EA0163D360D8E7884A30
:1022EC00136823F080031360FEF7F8FA0546844B5D
:1022FC001B6813F4807FCBD0FEF7F0FA401B02284A
:10230C00F5D90320B1E17E4A536F23F001035367E3
:10231C00FEF7E4FA05467A4B5B6F13F0020F06D01A
:10232C00FEF7DCFA401B0228F5D903209DE1236857
:10233C0013F0200F29D0A3699BB1714A136843F4A1
:10234C0080531360FEF7CAFA05466D4B1B6813F4F5
:10235C00005F1AD1FEF7C2FA401B0228F5D9032000
:10236C0083E1674A136823F480531360FEF7B6FACF
:10237C000546634B1B6813F4005F06D0FEF7AEFAFC
:10238C00401B0228F5D903206FE1236813F0040FDA
:10239C0022D1636A002B00F06781594A126902F05E
:1023AC003802182A00F00E81022B00F09480544A57
:1023BC00136823F080731360FEF790FA0446504BB9
:1023CC001B6813F0007F00F0FB80FEF787FA001B00
:1023DC000228F4D9032048E14A4A136843F4807375
:1023EC001360FEF77BFA0546464B1B6813F4807F9F
:1023FC0006D1FEF773FA401B6428F5D9032034E1AB
:10240C00A368012B0ED033BB3D4B1A6F22F0010297
:10241C001A671A6F22F080021A671A6F22F00402F0
:10242C001A6704E0364A136F43F001031367A3687D
:10243C00002B3ED0FEF752FA0546314B1B6F13F0C2
:10244C00020FA6D1FEF74AFA401B41F2883398429C
:10245C00F3D9032009E1052B0FD0852B1BD0284B7A
:10246C001A6F22F001021A671A6F22F004021A671F
:10247C001A6F22F080021A67D9E7214B1A6F42F0CB
:10248C0004021A671A6F22F080021A671A6F42F060
:10249C0001021A67CBE71A4B1A6F42F004021A6753
:1024AC001A6F42F080021A671A6F42F001021A6723
:1024BC00BDE7FEF713FA0546114B1B6F13F0020F25
:1024CC003FF467AFFEF70AFA401B41F2883398429B
:1024DC00F2D90320C9E00A4A136823F08073136011
:1024EC00FEF7FCF90546064B1B6813F0007F0BD07A
:1024FC00FEF7F4F9401B0228F5D90320B5E000BF24
:10250C0000440258004802585F4B996A5F4A0A40DF
:10251C00A16AE06A41EA00110A439A62226B013A0D
:10252C00C2F30802616B0139490289B20A43A16BFB
:10253C000139090401F4FE010A43E16B0139090672
:10254C0001F0FE410A431A63DA6A22F00102DA62F0
:10255C005A6B6FF3CF02A16C42EAC1025A63DA6A7A
:10256C0022F00C02216C0A43DA62DA6A22F00202CF
:10257C00616C0A43DA62DA6A42F48032DA62DA6A4D
:10258C0042F40032DA62DA6A42F48022DA62DA6AFF
:10259C0042F00102DA621A6842F080721A60FEF7A9
:1025AC009DF90446384B1B6813F0007F06D1FEF7EB
:1025BC0095F9001B0228F5D9032056E0002054E0C1
:1025CC00002052E030498A6A086B012B4ED002F091
:1025DC000303A16A8B424BD1C2F30512E36A9A4200
:1025EC0048D1C0F30802236B013B9A4244D1C0F39B
:1025FC004622636B013B9A4240D1C0F30642A36B67
:10260C00013B9A423CD1C0F30660E36B013B98421C
:10261C0038D11D4B5B6BC3F3CC03A26C9A4201D136
:10262C00002022E0184AD36A23F00103D362FEF79C
:10263C0055F90546FEF752F9A842FBD0124A536BE6
:10264C006FF3CF03A16C43EAC1035363D36A43F026
:10265C000103D362002008E001207047012004E050
:10266C00012002E0012000E0002038BD0120FCE741
:10267C000120FAE70120F8E70120F6E70120F4E752
:10268C000120F2E70120F0E7004402580CFCFFFFA8
:10269C00754B1B6903F03803102B00F0DE80182BF0
:1026AC000FD0002B40F0DB806F4B1B6813F0200F1A
:1026BC0000F0D7806C4B1B68C3F3C1036B48D84048
:1026CC00704710B4684B9A6A02F003029C6AC4F318
:1026DC000510D96A01F001015B6BC3F3CC0301FB5C
:1026EC0003F307EE903AF8EE677A14F47C7F77D018
:1026FC00012A4AD0022A76D0002A40F091805A4B07
:10270C001B6813F0200F23D057490A68C2F3C1028B
:10271C00564BD34007EE103AF8EE476A07EE100A14
:10272C00B8EE476A86EE867A0B6BC3F3080306EEA7
:10273C00903AF8EE666A9FED4E6A67EE867A76EE10
:10274C00A77AF7EE006A77EEA67A27EE277A38E0BA
:10275C0007EE100AF8EE476A9FED466A86EE267A77
:10276C00414B1B6BC3F3080306EE903AF8EE666A16
:10277C009FED3F6A67EE867A76EEA77AF7EE006AEF
:10278C0077EEA67A27EE277A1BE007EE100AF8EE12
:10279C00476A9FED396A86EE267A334B1B6BC3F37F
:1027AC00080306EE903AF8EE666A9FED316A67EE22
:1027BC00867A76EEA77AF7EE006A77EEA67A27EE9F
:1027CC00277A294B1B6BC3F34623013307EE903A50
:1027DC00F8EE677AC7EE276AFCEEE67A17EE900AF7
:1027EC005DF8044B704707EE100AF8EE476A9FED50
:1027FC00236A86EE267A1C4B1B6BC3F3080306EE8A
:10280C00903AF8EE666A9FED1A6A67EE867A76EE73
:10281C00A77AF7EE006A77EEA67A27EE277AD0E74A
:10282C0007EE100AF8EE476A9FED136A86EE267AD9
:10283C000D4B1B6BC3F3080306EE903AF8EE666A79
:10284C009FED0B6A67EE867A76EEA77AF7EE006A52
:10285C0077EEA67A27EE277AB3E70948704709483E
:10286C0070470248704700BF004402580090D003E4
:10287C00000000390024744C0024744A0024744B6A
:10288C000024F40000093D00002800F0328170B5EE
:10289C000D4604469B4B1B6803F00F038B420BD277
:1028AC00984A136823F00F030B431360136803F06B
:1028BC000F038B4240F01F81236813F0040F0CD0E0
:1028CC002269914B9B6903F070039A4205D98E499A
:1028DC008B6923F070031A438A61236813F0080F85
:1028EC000CD06269884BDB6903F070039A4205D9FE
:1028FC008549CB6923F070031A43CA61236813F02E
:10290C00100F0CD0A269804BDB6903F4E0639A4290
:10291C0005D97D49CB6923F4E0631A43CA61236866
:10292C0013F0200F0CD0E269774B1B6A03F0700395
:10293C009A4205D974490B6A23F070031A430A6250
:10294C00236813F0020F0CD0E2686F4B9B6903F005
:10295C000F039A4205D96C498B6923F00F031A4374
:10296C008A61236813F0010F41D0674A936923F4FD
:10297C007063A1680B4393616368022B0AD0032B2D
:10298C0027D0012B2CD0604A126812F0040F06D10C
:10299C000120ADE0126812F4003F00F0AE805A49FD
:1029AC000A6922F0070213430B61FDF797FF0646F5
:1029BC00554B1B6903F038036268B3EBC20F16D09A
:1029CC00FDF78CFF801B41F288339842F0D903202D
:1029DC008EE04D4A126812F0007FE0D1012087E0B2
:1029EC00494A126812F4807FD9D1012080E0236813
:1029FC0013F0020F0CD0E268434B9B6903F00F03FA
:102A0C009A4205D240498B6923F00F031A438A611D
:102A1C003C4B1B6803F00F03AB420AD9394A1368CD
:102A2C0023F00F032B431360136803F00F03AB4227
:102A3C0065D1236813F0040F0CD02269324B9B69CB
:102A4C0003F070039A4205D22F498B6923F070036F
:102A5C001A438A61236813F0080F0CD062692A4B61
:102A6C00DB6903F070039A4205D22749CB6923F046
:102A7C0070031A43CA61236813F0100F0CD0A269BB
:102A8C00214BDB6903F4E0639A4205D21E49CB6902
:102A9C0023F4E0631A43CA61236813F0200F0CD0AF
:102AAC00E269194B1B6A03F070039A4205D216496E
:102ABC000B6A23F070031A430A62FFF7E9FD12490F
:102ACC008B69C3F30323114AD35C03F01F03D84073
:102ADC008B6903F00F03D35C03F01F0320FA03F39D
:102AEC000B4A13600B4B18600B4B1868FDF794FEE8
:102AFC0070BD012070470120FAE70120F8E70120A2
:102B0C00F6E700BF0020005200440258EC4D0008CC
:102B1C00080000200C0000200400002008B5FFF77E
:102B2C00B7FD0B4A9369C3F303230A49CB5C03F04B
:102B3C001F0320FA03F3926902F00F02885C00F085
:102B4C001F0023FA00F0044A1060044A136008BD09
:102B5C0000440258EC4D0008080000200C00002036
:102B6C0008B5FFF7DBFF054BDB69C3F30213044A1F
:102B7C00D35C03F01F03D84008BD00BF00440258CB
:102B8C00EC4D0008404B9B6A03F00303032B79D0F8
:102B9C0070B505460E463C4A136823F080631360FB
:102BAC00FDF79CFE0446384B1B6813F0006F06D0F3
:102BBC00FDF794FE031B022BF5D9032070BD324B9D
:102BCC009A6A22F47C32296842EA01329A626A6873
:102BDC00013AC2F30802A9680139490289B20A43D1
:102BEC00E9680139090401F4FE010A432969013934
:102BFC00090601F0FE410A439A63DA6A22F0C00228
:102C0C0069690A43DA62DA6A22F02002A9690A4386
:102C1C00DA62DA6A22F01002DA62DA6B6FF3CF0250
:102C2C00E96942EAC102DA63DA6A42F01002DA6256
:102C3C00C6B91A46DB6A43F40023D362124A1368FE
:102C4C0043F080631360FDF749FE04460E4B1B688E
:102C5C0013F0006F14D1FDF741FE001B0228F5D9CB
:102C6C000320ABE7012E05D0074AD36A43F40013C7
:102C7C00D362E3E7044AD36A43F48013D362DDE7FB
:102C8C0000209BE70120704700440258404B9B6A90
:102C9C0003F00303032B79D070B505460E463C4A6E
:102CAC00136823F080531360FDF718FE0446384B6D
:102CBC001B6813F0005F06D0FDF710FE031B022B00
:102CCC00F5D9032070BD324B9A6A22F07C722968C8
:102CDC0042EA01529A626A68013AC2F30802A96890
:102CEC000139490289B20A43E9680139090401F43E
:102CFC00FE010A4329690139090601F0FE410A4324
:102D0C001A64DA6A22F4406269690A43DA62DA6A9E
:102D1C0022F40072A9690A43DA62DA6A22F4807238
:102D2C00DA625A6C6FF3CF02E96942EAC1025A6463
:102D3C00DA6A42F48072DA62C6B91A46DB6A43F484
:102D4C008003D362124A136843F080531360FDF77B
:102D5C00C5FD04460E4B1B6813F0005F14D1FDF744
:102D6C00BDFD001B0228F5D90320ABE7012E05D0D1
:102D7C00074AD36A43F08073D362E3E7044AD36A09
:102D8C0043F40003D362DDE700209BE7012070478A
:102D9C0000440258F8B50446036813F0006F30D0B5
:102DAC00C36EB3F5001F26D00ED8ABB1B3F5801FA0
:102DBC0007D102210830FFF7E5FE054695B12E46F6
:102DCC0021E0012635461EE0B3F5401F01D1002558
:102DDC0008E00126354616E0974AD36A43F40033DF
:102DEC00D3620025944A136D23F44013E16E0B4318
:102DFC001365002607E002212830FFF747FF054640
:102E0C00DCE700263546236813F4807F14D0A36DCD
:102E1C00042B31D8DFE803F0032229080800864A86
:102E2C00D36A43F40033D3624DBB834A136D23F052
:102E3C000703A16D0B431365236813F4007F42D085
:102E4C00E36D802B31D01FD84BB3402B19D100210F
:102E5C0004F10800FFF796FE05462CE0002104F172
:102E6C000800FFF78FFE0546DEE7002104F128007D
:102E7C00FFF70CFF0546D7E701263546DCE72E4663
:102E8C00DAE7012635461EE0B3F5807F13D0B3F5A3
:102E9C00A07F10D0C02B0ED00126354613E0664A19
:102EAC00D36A43F40033D36205E0002104F1280017
:102EBC00FFF7ECFE0546D5B95F4A136D23F4E073BA
:102ECC00E16D0B431365236813F4806F34D0236ECC
:102EDC00B3F5806F22D00FD8D3B1B3F5007F08D1F2
:102EEC00002104F10800FFF74DFE05461CE02E46BC
:102EFC00E9E7012635461FE0B3F5006F14D0B3F5B2
:102F0C00206F11D0B3F5C06F0ED00126354613E0FB
:102F1C00494AD36A43F40033D36205E0002104F13B
:102F2C002800FFF7B3FE0546BDB9434A136D23F4E1
:102F3C006063216E0B431365236813F0007F24D06C
:102F4C00E36C202B13D00DD8BBB1102B07D13A4A10
:102F5C00D36A43F40033D3620FE02E46ECE701262C
:102F6C00354612E0302B08D0012635460DE0022103
:102F7C0004F10800FFF706FE0546D5B92E4AD36CBE
:102F8C0023F03003E16C0B43D364236813F4805FAC
:102F9C0031D0636EB3F5005F1FD00FD8BBB1B3F562
:102FAC00805F08D1002104F10800FFF7EBFD054616
:102FBC0019E02E46E9E7012635461CE0B3F5405FE3
:102FCC0011D0B3F5804F0ED00126354613E01A4AC6
:102FDC00D36A43F40033D36205E0002104F12800E6
:102FEC00FFF754FE054615BB134A136D23F4E0435B
:102FFC00616E0B431365236813F4005F32D0A36E2C
:10300C00B3F5003F26D019D843B1B3F5803F10D1AA
:10301C00012104F10800FFF7B5FD05460DBB064A7A
:10302C00136D23F4E023A16E0B4313651AE02E46B7
:10303C00E1E70126354615E000440258B3F5802F30
:10304C00ECD0B3F5A02FE9D0B3F5403FE6D0012684
:10305C00354607E0012104F12800FFF717FE05466D
:10306C00DCE72E46236813F4804F18D0D4F8B03028
:10307C00B3F1005F38D024D843B1B3F1805F1DD1D8
:10308C00012104F10800FFF77DFD05469DBB904A28
:10309C00936D23F0E043D4F8B0100B439365236891
:1030AC0013F4004F3FD0A36FB3F1805F25D0B3F181
:1030BC00005F30D033B30126354634E00126354667
:1030CC00EDE7B3F1A04FE1D008D8B3F1405FDDD00C
:1030DC00B3F1804FDAD001263546E0E7B3F1C04FAB
:1030EC00D4D001263546DAE7012104F12800FFF798
:1030FC00CDFD0546CAE72E46D1E7754AD36A43F49F
:10310C000033D36275B9724A136D23F04053A16F2B
:10311C000B43136507E0012104F10800FFF732FDB2
:10312C000546EFE72E46236813F0807F13D0A36C7F
:10313C00032B3CD8DFE803F007023407644AD36A58
:10314C0043F40033D362ADBB614AD36C23F0030369
:10315C00A16C0B43D364236813F4800F2CD1236828
:10316C0013F0010F00F0A580D4F88430282B00F266
:10317C009E80DFE803F08B9C9C9C9C9C9C9C859C7B
:10318C009C9C9C9C9C9C959C9C9C9C9C9C9C8B9C8B
:10319C009C9C9C9C9C9C8B9C9C9C9C9C9C9C8B0021
:1031AC00022104F10800FFF7EDFC0546CBE70126F0
:1031BC003546D0E72E46CEE7464A136843F4807373
:1031CC001360FDF78BFB0746424B1B6813F4807FA3
:1031DC0005D1FDF783FBC01B6428F5D90325002D11
:1031EC004AD13B4B1B6FD4F8B420534013F4407FAF
:1031FC000CD0374B1A6F22F44072196F41F48031A6
:10320C001967196F21F4803119671A67D4F8B43033
:10321C00B3F5807F15D08DBBD4F8B43003F4407275
:10322C00B2F5407F1ED02A4A136923F47C531361F4
:10323C0027490B6FD4F8B420C2F30B0213430B676E
:10324C008DE7FDF74BFB0746214B1B6F13F0020F6D
:10325C00E1D1FDF743FBC01B41F288339842F3D90F
:10326C000325D8E71A48026922F47C521A4901EA6C
:10327C00131313430361DBE72E4670E72E466EE70C
:10328C00012104F10800FFF77DFC0546F5B9104A51
:10329C00536D23F03803D4F884100B43536508E0C6
:1032AC00012104F12800FFF7F1FC0546EEE70126A9
:1032BC003546236813F0020F1FD0D4F88030052B4D
:1032CC0033D8DFE803F0110B2B1111112E46F0E768
:1032DC000044025800480258CFFFFF00012104F1BE
:1032EC000800FFF74FFC054615BBB74A536D23F09A
:1032FC000703D4F880100B435365236813F0040FB5
:10330C0029D0D4F89C30052B00F20881DFE813F0AB
:10331C0018001200FF00180018001800012104F119
:10332C002800FFF7B3FC0546DEE701263546E4E747
:10333C002E46E2E7012104F10800FFF723FC0546C5
:10334C00002D40F0EE80A04A936D23F00703D4F8D3
:10335C009C100B439365236813F0200F1DD0D4F8F9
:10336C009830B3F1005F00F0F08000F2DF804BB1D9
:10337C00B3F1805F40F0D780002104F10800FFF723
:10338C0001FC0546002D40F0E7808F4A536D23F079
:10339C00E043D4F898100B435365236813F0400FA7
:1033AC001DD0D4F8A430B3F5006F00F0E98000F222
:1033BC00D8804BB1B3F5806F40F0D080002104F180
:1033CC000800FFF7DFFB0546002D40F0E0807E4A49
:1033DC00936D23F4E053D4F8A4100B439365236846
:1033EC0013F0800F1DD0D4F8A830B3F5804F00F047
:1033FC00E28000F2D1804BB1B3F5005F40F0C980A0
:10340C00002104F10800FFF7BDFB0546002D40F03C
:10341C00D9806D4A936D23F46043D4F8A8100B4304
:10342C009365236813F0080F0DD0D4F88C30B3F5E6
:10343C00805F00F0CB80644A536D23F44053D4F882
:10344C008C100B435365236813F0100F0DD0D4F878
:10345C00A030B3F5807F00F0C3805B4A936D23F4FA
:10346C004073D4F8A0100B439365236813F4002F1A
:10347C001CD0D4F8AC30B3F5803F00F0BB80B3F572
:10348C00003F08D0002B40F0BC80002104F1080064
:10349C00FFF778FB0546002D40F0B6804A4A936D45
:1034AC0023F44033D4F8AC100B439365236813F426
:1034BC00802F1CD0D4F89030B3F5001F00F0A680FC
:1034CC00B3F5401F08D0B3F5801F40F0A6803E4AEC
:1034DC00D36A43F40033D362002D40F0A1803A4A02
:1034EC00536D23F44013D4F890100B4353652368A9
:1034FC0013F4803F00F0AC80236D002B00F0928021
:10350C00B3F5803F00F09C8001263546A0E00121F8
:10351C0004F12800FFF7BAFB054611E701263546F2
:10352C0019E72E4617E70126354636E7B3F1804FEB
:10353C003FF428AFB3F1A04F3FF424AFB3F1405F99
:10354C003FF420AF0126354627E7022104F128007D
:10355C00FFF79CFB054615E72E461EE70126354670
:10356C003DE7B3F5805F3FF42FAFB3F5A05F3FF4B9
:10357C002BAFB3F5406F3FF427AF012635462EE74E
:10358C00022104F12800FFF781FB05461CE72E46BB
:10359C0025E70126354644E7B3F5004F3FF436AF37
:1035AC00B3F5204F3FF432AFB3F5C04F3FF42EAF1D
:1035BC000126354635E7022104F12800FFF766FBAA
:1035CC00054623E72E462CE700440258022104F15D
:1035DC002800FFF75BFB00283FF42DAF01262AE7FC
:1035EC00022104F12800FFF751FB00283FF435AF0E
:1035FC00012632E7022104F12800FFF747FB0546BC
:10360C0049E70126354651E72E464FE7012104F1E3
:10361C002800FFF73BFB05465EE70126354666E7CB
:10362C002E4664E76F4AD36A43F40033D36275B90C
:10363C006C4AD36C23F48033216D0B43D36407E0C5
:10364C00022104F10800FFF79DFA0546EFE72E462C
:10365C00236813F0005F11D1236813F4003F28D0C6
:10366C00D4F88830B3F5807F14D010D9B3F5007F2F
:10367C0015D0B3F5407F12D001261AE0022104F1D7
:10368C002800FFF703FB0028E6D00126E4E733B15E
:10369C0001260EE0534AD36A43F40033D362002D63
:1036AC0068D1504A536D23F44073D4F888100B43FF
:1036BC005365236813F4801F06D04A4A136D23F018
:1036CC000043E16F0B431365236813F4001F06D00E
:1036DC00444A136D23F08073216F0B4313652368E9
:1036EC0013F4006F06D03F4A936D23F00063616FB3
:1036FC000B439365236813F0804F09D0394B1A693B
:10370C0022F400421A611A69D4F8B8100A431A61FB
:10371C002368002B06DA334AD36C23F04053616DD7
:10372C000B43D364236813F4000F07D02D4A536D59
:10373C0023F44003D4F894100B435365636813F0DF
:10374C00010F19D1636813F0020F1ED1636813F0D7
:10375C00040F23D1636813F0080F28D1636813F0AA
:10376C00100F2DD1636813F0200F32D106B1012652
:10377C003046F8BD2E469CE7002104F10800FFF707
:10378C0001FA0028DED00646DCE7012104F108002E
:10379C00FFF7F8F90028D9D00646D7E7022104F143
:1037AC000800FFF7EFF90028D4D00646D2E7002135
:1037BC0004F12800FFF76AFA0028CFD00646CDE7BF
:1037CC00012104F12800FFF761FA0028CAD006464F
:1037DC00C8E7022104F12800FFF758FA0028C5D0E9
:1037EC000126C5E70044025808B5FFF797F9054BC9
:1037FC001B6AC3F30213044AD35C03F01F03D840C3
:10380C0008BD00BF00440258EC4D000810B4794BC1
:10381C009A6A9C6AC4F3053CD96AC1F30011DB6B4C
:10382C00C3F3CC0301FB03F314F47C3F00F0DD8005
:10383C0002F0030207EE903AF8EE677A012A4BD0B9
:10384C00022A00F09880002A40F0B280694B1B6875
:10385C0013F0200F23D067490A68C2F3C102664BEC
:10386C00D34007EE103AF8EE476A07EE10CAB8EEEE
:10387C00476A86EE867A8B6BC3F3080306EE903AA2
:10388C00F8EE666A9FED5D6A67EE867A76EEA77A49
:10389C00F7EE006A77EEA67A27EE277A38E007EE85
:1038AC0010CAF8EE476A9FED566A86EE267A514B9F
:1038BC009B6BC3F3080306EE903AF8EE666A9FED35
:1038CC004F6A67EE867A76EEA77AF7EE006A77EEA5
:1038DC00A67A27EE277A1BE007EE10CAF8EE476AA5
:1038EC009FED486A86EE267A424B9B6BC3F3080326
:1038FC0006EE903AF8EE666A9FED406A67EE867ABD
:10390C0076EEA77AF7EE006A77EEA67A27EE277A9C
:10391C00384A936BC3F3462307EE903AF8EE677A76
:10392C00F7EE006A77EEA67A87EE276ABCEEC66AD7
:10393C0080ED006A936BC3F3064307EE903AF8EE02
:10394C00677A77EEA67A87EE276ABCEEC66A80EDB8
:10395C00016A936BC3F3066307EE903AF8EE677A4D
:10396C0077EEA67AC7EE276AFCEEE66AC0ED026A2D
:10397C005DF8044B704707EE10CAF8EE476A9FEDEE
:10398C00226A86EE267A1B4B9B6BC3F3080306EE6A
:10399C00903AF8EE666A9FED196A67EE867A76EED3
:1039AC00A77AF7EE006A77EEA67A27EE277AAFE7CA
:1039BC0007EE10CAF8EE476A9FED126A86EE267A79
:1039CC000C4B9B6BC3F3080306EE903AF8EE666A59
:1039DC009FED0A6A67EE867A76EEA77AF7EE006AB2
:1039EC0077EEA67A27EE277A92E7002303604360EE
:1039FC008360BDE7004402580090D00300000039FA
:103A0C000024744C0024744A0024744B10B4794B79
:103A1C009A6A9C6AC4F3055CD96AC1F300215B6C99
:103A2C00C3F3CC0301FB03F314F07C7F00F0DD80C7
:103A3C0002F0030207EE903AF8EE677A012A4BD0B7
:103A4C00022A00F09880002A40F0B280694B1B6873
:103A5C0013F0200F23D067490A68C2F3C102664BEA
:103A6C00D34007EE103AF8EE476A07EE10CAB8EEEC
:103A7C00476A86EE867A0B6CC3F3080306EE903A1F
:103A8C00F8EE666A9FED5D6A67EE867A76EEA77A47
:103A9C00F7EE006A77EEA67A27EE277A38E007EE83
:103AAC0010CAF8EE476A9FED566A86EE267A514B9D
:103ABC001B6CC3F3080306EE903AF8EE666A9FEDB2
:103ACC004F6A67EE867A76EEA77AF7EE006A77EEA3
:103ADC00A67A27EE277A1BE007EE10CAF8EE476AA3
:103AEC009FED486A86EE267A424B1B6CC3F30803A3
:103AFC0006EE903AF8EE666A9FED406A67EE867ABB
:103B0C0076EEA77AF7EE006A77EEA67A27EE277A9A
:103B1C00384A136CC3F3462307EE903AF8EE677AF3
:103B2C00F7EE006A77EEA67A87EE276ABCEEC66AD5
:103B3C0080ED006A136CC3F3064307EE903AF8EE7F
:103B4C00677A77EEA67A87EE276ABCEEC66A80EDB6
:103B5C00016A136CC3F3066307EE903AF8EE677ACA
:103B6C0077EEA67AC7EE276AFCEEE66AC0ED026A2B
:103B7C005DF8044B704707EE10CAF8EE476A9FEDEC
:103B8C00226A86EE267A1B4B1B6CC3F3080306EEE7
:103B9C00903AF8EE666A9FED196A67EE867A76EED1
:103BAC00A77AF7EE006A77EEA67A27EE277AAFE7C8
:103BBC0007EE10CAF8EE476A9FED126A86EE267A77
:103BCC000C4B1B6CC3F3080306EE903AF8EE666AD6
:103BDC009FED0A6A67EE867A76EEA77AF7EE006AB0
:103BEC0077EEA67A27EE277A92E7002303604360EC
:103BFC008360BDE7004402580090D00300000039F8
:103C0C000024744C0024744A0024744B10B4794B77
:103C1C009A6A9C6AC4F3051CD96A01F001015B6BBA
:103C2C00C3F3CC0301FB03F314F47C7F00F0DD80C1
:103C3C0002F0030207EE903AF8EE677A012A4BD0B5
:103C4C00022A00F09880002A40F0B280694B1B6871
:103C5C0013F0200F23D067490A68C2F3C102664BE8
:103C6C00D34007EE103AF8EE476A07EE10CAB8EEEA
:103C7C00476A86EE867A0B6BC3F3080306EE903A1E
:103C8C00F8EE666A9FED5D6A67EE867A76EEA77A45
:103C9C00F7EE006A77EEA67A27EE277A38E007EE81
:103CAC0010CAF8EE476A9FED566A86EE267A514B9B
:103CBC001B6BC3F3080306EE903AF8EE666A9FEDB1
:103CCC004F6A67EE867A76EEA77AF7EE006A77EEA1
:103CDC00A67A27EE277A1BE007EE10CAF8EE476AA1
:103CEC009FED486A86EE267A424B1B6BC3F30803A2
:103CFC0006EE903AF8EE666A9FED406A67EE867AB9
:103D0C0076EEA77AF7EE006A77EEA67A27EE277A98
:103D1C00384A136BC3F3462307EE903AF8EE677AF2
:103D2C00F7EE006A77EEA67A87EE276ABCEEC66AD3
:103D3C0080ED006A136BC3F3064307EE903AF8EE7E
:103D4C00677A77EEA67A87EE276ABCEEC66A80EDB4
:103D5C00016A136BC3F3066307EE903AF8EE677AC9
:103D6C0077EEA67AC7EE276AFCEEE66AC0ED026A29
:103D7C005DF8044B704707EE10CAF8EE476A9FEDEA
:103D8C00226A86EE267A1B4B1B6BC3F3080306EEE6
:103D9C00903AF8EE666A9FED196A67EE867A76EECF
:103DAC00A77AF7EE006A77EEA67A27EE277AAFE7C6
:103DBC0007EE10CAF8EE476A9FED116A86EE267A76
:103DCC000C4B1B6BC3F3080306EE903AF8EE666AD5
:103DDC009FED0A6A67EE867A76EEA77AF7EE006AAE
:103DEC0077EEA67A27EE277A92E7002303604360EA
:103DFC008360BDE7004402580090D00300000039F6
:103E0C000024744C0024744A0024744B00B58BB00D
:103E1C00A0F580730B4328D0A0F500730B4377D02B
:103E2C00A0F580630B4300F0CB80A0F580530B43CF
:103E3C0000F02381A0F500530B4300F08381A0F523
:103E4C0000230B4300F0CC81A0F580330B4300F032
:103E5C000F82A0F580430B4300F02882A0F50040B0
:103E6C00084300F07D8200200CE0944B1B6D03F0A6
:103E7C000703042B00F29E82DFE803F007111B03FB
:103E8C0025008F480BB05DF804FB8C4B186810F0C4
:103E9C000070F7D007A8FFF7B9FE0898F2E7874B38
:103EAC00186810F00060EDD004A8FFF7AFFC049880
:103EBC00E8E7824B186810F00050E3D001A8FFF738
:103ECC00A5FD0198DEE77D4AD36C03F040531268E0
:103EDC0012F0040F07D033B9784B1B68C3F3C1033E
:103EEC007848D840CEE7754A126812F4807F03D028
:103EFC00B3F1805F00F06082704A126812F4003FE8
:103F0C0000F05C82B3F1005F00F05A820020B9E748
:103F1C006A4B1B6D03F4E073802B31D015D9C02B89
:103F2C0000F05082B3F5807F1ED1644AD36C03F04D
:103F3C004053126812F0040F2DD063BB5F4B1B680B
:103F4C00C3F3C1035F48D8409CE77BB1402B09D138
:103F5C005A4B186810F0006094D004A8FFF756FC78
:103F6C0004988FE700208DE700208BE7534B1868EF
:103F7C0010F0007086D007A8FFF748FE089881E77C
:103F8C004E4B186810F000503FF47CAF01A8FFF7BF
:103F9C003DFD019876E7494A126812F4807F03D000
:103FAC00B3F1805F00F01082444A126812F4003FB3
:103FBC0000F00C82B3F1005F00F00A82002061E790
:103FCC003E4B1B6D03F46063B3F5806F35D016D98F
:103FDC00B3F5C06F00F0FE81B3F5006F20D1374A06
:103FEC00D36C03F04053126812F0040F30D07BBB3B
:103FFC00324B1B68C3F3C1033248D84042E78BB144
:10400C00B3F5007F0AD12D4B186810F000603FF417
:10401C0039AF04A8FFF7FAFB049833E7002031E727
:10402C0000202FE7254B186810F000703FF42AAFE2
:10403C0007A8FFF7EBFD089824E7204B186810F051
:10404C0000503FF41FAF01A8FFF7E0FC019819E7FF
:10405C001A4A126812F4807F03D0B3F1805F00F02B
:10406C00BB81164A126812F4003F00F0B781B3F11D
:10407C00005F00F0B581002004E7104B1B6D03F4CA
:10408C00E043B3F5005F3DD01ED9B3F5405F00F0BF
:10409C00A981B3F5804F28D1084AD36C03F0405363
:1040AC00126812F0040F38D0002B36D1034B1B686A
:1040BC00C3F3C1030348D840E4E600BF00440258F0
:1040CC000080BB000090D0038BB1B3F5805F0AD1A8
:1040DC009F4B186810F000603FF4D4AE04A8FFF7B3
:1040EC0095FB0498CEE60020CCE60020CAE6984B5F
:1040FC00186810F000703FF4C5AE07A8FFF786FDF6
:10410C000898BFE6924B186810F000503FF4BAAE16
:10411C0001A8FFF77BFC0198B4E68D4A126812F4F3
:10412C00807F03D0B3F1805F00F05E81884A126813
:10413C0012F4003F00F05A81B3F1005F00F0588197
:10414C0000209FE6824B1B6D03F4E023B3F5403F48
:10415C0032D00BD8B3F5803F18D0B3F5003F20D048
:10416C0013B9FEF7FDFC8DE600208BE6B3F5802F2E
:10417C002ED0B3F5A02F07D1754B186810F4003072
:10418C003FF480AE73487DE600207BE6704B1868E8
:10419C0010F000603FF476AE04A8FFF737FB0598EB
:1041AC0070E66B4B186810F000503FF46BAE01A832
:1041BC00FFF72CFC029865E6654B186810F00400BC
:1041CC003FF460AE1B68C3F3C1036348D84059E6A3
:1041DC005F4B186810F480703FF454AE5F4851E6A2
:1041EC005B4B9B6D03F44033B3F5803F10D0B3F5BC
:1041FC00003F18D0002B40F0FD80554B186810F094
:10420C0000603FF43FAE04A8FFF700FB049839E6CA
:10421C004F4B186810F000503FF434AE01A8FFF774
:10422C00F5FB03982EE64A4AD36C03F04053126810
:10423C0012F0040F07D033B9454B1B68C3F3C1030D
:10424C004548D8401EE6424A126812F4807F03D0DB
:10425C00B3F1805F00F0D0803D4A126812F4003F49
:10426C0000F0CC80B3F1005F00F0CA80002009E6BA
:10427C00374BDB6C13F4803302D063B9002001E6BA
:10428C00334B186810F000703FF4FCAD07A8FFF733
:10429C00BDFC0898F6E52E4B186810F000603FF452
:1042AC00F1AD04A8FFF7B2FA0698EBE5284B9B6D2D
:1042BC0003F0E043B3F1405F36D00BD8B3F1805F2D
:1042CC001CD0B3F1005F24D013B9FFF78DFAD9E5F8
:1042DC000020D7E5B3F1A04F32D0B3F1C04F00F0BE
:1042EC009180B3F1804F07D1194B186810F480708E
:1042FC003FF4C8AD1948C5E50020C3E5144B186858
:10430C0010F000603FF4BEAD04A8FFF77FFA0598EB
:10431C00B8E50F4B186810F000503FF4B3AD01A88E
:10432C00FFF774FB0298ADE5094B186810F0040018
:10433C003FF4A8AD1B68C3F3C1030748D840A1E5FF
:10434C00034B186810F400303FF49CAD014899E51C
:10435C00004402580024F4000090D00300093D00F2
:10436C002A4B1B6D03F04053B3F1805F0CD0B3F1BB
:10437C00005F14D0002B47D1244B186810F4003088
:10438C003FF480AD22487DE5204B186810F000709A
:10439C003FF478AD07A8FFF739FC089872E51B4B82
:1043AC00186810F000603FF46DAD04A8FFF72EFA0A
:1043BC00059867E5002065E5164863E5002061E592
:1043CC0013485FE514485DE512485BE5002059E5AC
:1043DC000F4857E5104855E50E4853E5002051E5C8
:1043EC000B484FE50C484DE50A484BE5002049E5E4
:1043FC00074847E5002045E5064843E5002041E530
:10440C0003483FE504483DE500203BE500440258E5
:10441C000024F40000093D000080BB00C36B5B0965
:10442C00C0680830C00803FB00007047002800F08B
:10443C00B78070B504460023836205685C4B5D4E03
:10444C009D4218BFB54214BF0126002607D0A3F524
:10445C0074439D4203D0C3680F2B00F2A380204607
:10446C00FFF7DCFF2EB1544B9D4202D0082800F21E
:10447C009B804F4A4F4B9D4218BF954203D003F58A
:10448C0080639D4202D1102800F2908094F8813014
:10449C00F3B1022384F881302268136823F00103FE
:1044AC00136023689A6802F4F812A169B1F1806F65
:1044BC0014D0636813F4800F23D0E368062B20D943
:1044CC0021680B6823F48073206D03430B601DE09F
:1044DC0084F880302046FDF775FCDAE76168B1F5A9
:1044EC00800F06D00029E4D1A16BB1F1805FE0D13F
:1044FC0002E0A06B0028F5D1196841F480511960D5
:10450C00D7E721680B6823F480730B60E369A16A19
:10451C000B431343E26B1343E16822680B43936034
:10452C00636B626A1343A26B1343A2691343226940
:10453C00134362691343226A134362681343E26CA8
:10454C001343A2681343A26C1343A16D22680B435F
:10455C00D36063686BB92268936823F4C05343F447
:10456C00006393602268936823F4C06343F4806310
:10457C0093602268136D23F001031365636813F4D1
:10458C00800F06D02268D36823F00043616D0B4383
:10459C00D3600020C4F88400012384F8813070BDFE
:1045AC00012070470120FAE70120F8E70120F6E727
:1045BC000030014000380040003C004010B4036A59
:1045CC00046A24F001040462846924F0F00C4CEABF
:1045DC00021223F00A030B43826103625DF8044B61
:1045EC00704730B4056A046A24F0100404628469CC
:1045FC0024F4407C4CEA022C2CF4704C1B039BB230
:10460C0043EA0C0325F0A005090101F0A0012943A0
:10461C008361016230BC704710B4036A046A24F0F1
:10462C0010040462846924F4704C4CEA023223F0C6
:10463C00A00343EA0113826103625DF8044B7047E7
:10464C0030B4056A046A24F480740462C46924F0EA
:10465C00030C4CEA020C2CF0F00C1B01DBB243EA0D
:10466C000C0325F42065090201F420612943C36180
:10467C00016230BC704730B4056A046A24F480547B
:10468C000462C46924F4407C4CEA022C2CF4704C77
:10469C001B039BB243EA0C0325F42045090301F4E8
:1046AC0020412943C361016230BC704730B50368B7
:1046BC003D4A904214BF4FF0000E4FF0010EB0F186
:1046CC00804F14BF72464EF00102AAB9374CA0427B
:1046DC0014BF00240124364DA8420DD064B904F156
:1046EC00804404F58234A04214BF0024012405F553
:1046FC000065A84200D01CB123F070034C68234322
:10470C0012BB2A4A904214BF00220122284CA0421C
:10471C001AD0CAB902F1804202F58232904214BF1B
:10472C000022012204F50064A0420DD062B9214A96
:10473C00904214BF0022012204F59A34A04203D007
:10474C0012B91D4A904204D123F4407CCB6843EA51
:10475C000C0323F080034A69134303608A68C26226
:10476C000A688262154A904214BF73464EF00103E8
:10477C0063B9104B984214BF0023012302F5705209
:10478C00904203D013B90C4B984201D10B690363CF
:10479C0001234361036913F0010F03D0036923F074
:1047AC000103036130BD00BF000001400008004060
:1047BC000004004000440140004801400004014056
:1047CC0060B310B5044690F83D3013B3022384F85F
:1047DC003D30214651F8040BFFF768FF012384F8A4
:1047EC00483084F83E3084F83F3084F8403084F808
:1047FC00413084F8423084F8433084F8443084F8F3
:10480C00453084F8463084F8473084F83D30002039
:10481C0010BD80F83C30FDF7A9FBD7E701207047AD
:10482C0070B49446066A046A24F001040462846934
:10483C001D4DB0F1804F18BFA84223D01B4A9042A7
:10484C0014BF00220122A5F57C45A8421AD0CAB992
:10485C0002F1804202F58232904214BF0022012202
:10486C0005F50065A8420DD062B9114A904214BFFB
:10487C000022012205F54065A84203D012B944F08C
:10488C00010203E024F0030242EA0C0222F0F002DF
:10489C001B01DBB2134326F00A0201F00A0111439B
:1048AC008361016270BC7047000001400008004049
:1048BC000040014038B590F83C30012B5ED00446E6
:1048CC000D46012380F83C300C2A52D8DFE802F068
:1048DC0007515151195151512C5151513E00CB6836
:1048EC004A6809680068FFF79BFF2268936923F008
:1048FC000C03936122689369A9680B4393610020B0
:10490C0038E0CB684A6809680068FFF76AFE2268DD
:10491C00936923F44063936122689369A96843EA1D
:10492C0001239361002025E0CB684A680968006880
:10493C00FFF786FE2268D36923F00C03D36122684B
:10494C00D369A9680B43D361002013E0CB684A6894
:10495C0009680068FFF78FFE2268D36923F440636F
:10496C00D3612268D369A96843EA0123D36100208B
:10497C0000E00120002384F83C3038BD0220FCE725
:10498C0010B4846824F47F4C42EA03220A4342EABE
:10499C000C0282605DF8044B7047000010B504688F
:1049AC00A3684C4A1A404B6813434B4A1A400B6895
:1049BC001343A3604B68602B68D01ED8402B50D09B
:1049CC0008D9502B17D10A6989680068FFF7F6FDE2
:1049DC00002045E0202B60D007D8002B5FD0102B97
:1049EC0001D001203CE000203AE0302B01D0012026
:1049FC0036E0002034E0012032E0702B29D050D377
:104A0C00364A93424FD013D8303A93424DD007D9FF
:104A1C00334A93424FD0103293424ED100201FE0C4
:104A2C00B3F5801F43D0B3F1101F42D1002017E023
:104A3C00B3F5001F43D007D82A4A934241D0103215
:104A4C00934240D100200BE0274A93423DD10020F5
:104A5C0006E00B698A68C9680068FFF791FF0020BF
:104A6C0010BD0B68052B32D003681C6A1A6A22F041
:104A7C0001021A620268936923F0F003096943EAA0
:104A8C000113936103681C620020E9E70A698968D5
:104A9C000068FFF7C1FD0020E2E70020E0E70020FE
:104AAC00DEE70120DCE70020DAE70020D8E7002071
:104ABC00D6E70120D4E70020D2E70120D0E7002080
:104ACC00CEE70020CCE70120CAE70120C8E701208F
:104ADC00C6E700BF8FFFCFFFF8FFFEFF50001000AE
:104AEC0030001000600010001000200090F83C30E6
:104AFC00012B22D010B50446012380F83C30022350
:104B0C0080F83D30FFF74AFF80B92268D36823F064
:104B1C004003D3602268D36823F48043D36001231D
:104B2C0084F83D30002384F83C3010BD012084F81B
:104B3C003D00002384F83C30F7E70220704700006A
:104B4C0090F83C20012A45D070B40346012280F82D
:104B5C003C20022280F83D200268506894681E4E6A
:104B6C001E4DAA4218BFB24203D120F470004D680A
:104B7C00284320F070000D68284350601A681648CE
:104B8C00B2F1804F18BF824217D0A0F57C40824210
:104B9C0013D000F5806082420FD000F58060824215
:104BAC000BD000F57840824207D0A0F56C408242D1
:104BBC0003D000F59430824204D124F0800489683B
:104BCC0021439160012283F83D20002083F83C00B2
:104BDC0070BC704702207047000001400004014087
:104BEC00FEE7FEE7FEE7FEE7FEE77047704770471B
:104BFC0008B5FBF767FE08BD08B50248FCF778FD61
:104C0C0008BD00BF88010020224AD2F8883043F446
:104C1C007003C2F88830204B1B6803F00F03022B83
:104C2C0006D81D4A136823F00F0343F003031360E7
:104C3C001A4B1A6842F001021A6000221A611968B4
:104C4C00174A0A401A60144B1B6813F00C0F06D05D
:104C5C00114A136823F00F0343F0030313600F4B47
:104C6C0000229A61DA611A620E4999620E49D96280
:104C7C000E4919635A639963DA6319645A641968A3
:104C8C0021F4802119601A66094B43F2D2021A6092
:104C9C00704700BF00ED00E00020005200440258B5
:104CAC007FEDF6EA000202020000FF018002010122
:104CBC0000400052DFF834D0FFF7A6FF0C480D4936
:104CCC000D4A002302E0D458C4500433C4188C425B
:104CDC00F9D30A4A0A4C002301E013600432A242C1
:104CEC00FBD300F019F8FBF781FD704700000220A0
:104CFC000000002010000020044E000810000020CE
:104D0C00F8020020FEE702440346934200D17047AC
:104D1C0003F8011BF9E7000070B50D4B0D4D5B1B43
:104D2C009C100026A64209D100F028F80A4D0B4B26
:104D3C005B1B9C100026A64205D170BD55F8043BA8
:104D4C0098470136EEE755F8043B98470136F2E7F1
:104D5C00FC4D0008FC4D0008FC4D0008004E0008FE
:104D6C000A44914200F1FF3300D1704710B511F89D
:104D7C00014B03F8014F9142F9D110BDF8B500BFBA
:104D8C00F8BC08BC9E467047F8B500BFF8BC08BC20
:044D9C009E46704778
:104DA0000000000000000000000000000000000003
:104DB00000000000010000000200000003000000ED
:104DC00004000000000000000500000000000000DA
:104DD00000000000000000000600000000000000CD
:104DE00000000000000000000700000000000000BC
:0C4DF00001020304010203040607080985
:044DFC00D1020008D8
:044E0000AD020008F7
:104E040001000000100000000090D0030090D003C7
:0400000508004CC1E2
:00000001FF
